:10000000B601BB290408A7000610861086108316C7
:100010000610861086100F30860583122708B61842
:100020002F283A30A100983034213330A6004320E5
:100030001330A10088303421432064303321432021
:10004000643033212230A600432028302E200C308B
:100050002E2006302E20B61427082F283614A6008E
:10006000361C3D288610033C031C422842200730E2
:10007000A100D0303421031408003614FE3C0319CB
:10008000B6298614361C361006140F30860526084D
:10009000F03986040610A60E361843283230332174
:1000A000031408006400682003185228E020A80107
:1000B0000830A300E12068200318A80AAB1EA8019D
:1000C000A20CA30B5A28AB1AA213E12022080800A5
:1000D0003A088400380884178004841300052B1B19
:1000E0003806FF3E080029080319B629B121A903E3
:1000F0007328A401A501B712B121D33E0319B71685
:100100002D3EC63E03187C280A3E031C7C28A20014
:100110000310240DA000250DA100200DA10DA407A2
:100120000318A10A2108A507A40DA50D2208A407FC
:100130000318A50AA9030319A428B121C63E031870
:10014000A4280A3E03188728B71EAB28A409A509CE
:10015000A40A0319A50A2408B629A6003A088400AF
:10016000F030B7050830A70003100318B70AC620FF
:10017000A60CA70BB5280000AB1A370CC620B92176
:100180000314C6202F08A3002E0827298413AB1FB1
:10019000D528000838042B1F380680008417000873
:1001A0003804031C38068000E12800083804031CCA
:1001B00038062B1B38068000841738098005E12893
:1001C00037172B081F39FF3EA1002A08F53E0318F8
:1001D000A10A371F34293713A000023055213429D2
:1001E000A40029080319B6292408B121A903F1287C
:1001F000B71329080319B7170530A8002730A30043
:1002000010300E210330A300E8300E21A30164302A
:100210000E21A3010A300E2124081529A200250869
:10022000A1002408A0007F212008A000A803031932
:10023000B713290803191F292802031808002008EA
:10024000031DB713B71B0800303EB129A301A2005C
:10025000FF30A207031CA307031CB6290330A1002B
:10026000DF3034212829A101E83EA000A109FC309B
:10027000031C3D29A00703183A29A0076400A10F19
:100280003A2920184329A01C4729000047290800C3
:10029000A3015F21031950292308A1002208A0000F
:1002A000200808000310A10CA00CFF3E03185229DF
:1002B0002008B629A101A301A20002306829A200EA
:1002C00001306829A20006306829A200043068299C
:1002D000A80023082102031D6F29220820020430F0
:1002E00003180130031902302805031DFF30B62919
:1002F0000038031DFF300405031DFF30B629103000
:10030000A600A501A401210DA40DA50D2208A4029B
:100310002308031C230FA502031895292208A4070C
:1003200023080318230FA5070310A00DA10DA60B8A
:1003300083292008B6291030A800A101A001A70C2C
:10034000A60C031CA9292208A00723080318230FC1
:10035000A107A10CA00CA50CA40CA80B9F29240894
:10036000B629840031088A00300882008313031301
:100370008312640008000330A300E8308A012721BB
:1003800083161F30850086016F3087008312481462
:100390000714831607108312C901FE308A01032057
:1003A00001308A01032020308A01032020308A0195
:1003B000032050308A01032049308A010320433052
:1003C0008A0103202D308A01032054308A01032042
:1003D00043308A01032056308A01032052308A01BB
:1003E000032020308A01032031308A010320343079
:1003F0008A01032034308A01032020308A0103203F
:1004000020308A010320FE308A010320C0308A0197
:10041000032020308A01032020308A010320453048
:100420008A01032041308A01032033308A010320EE
:1004300043308A0103204E308A0103204F308A0165
:10044000032020308A01032020308A010320563007
:100450008A01032031308A0103202E308A010320D3
:1004600030308A01032020308A01032020308A01A5
:1004700003200730A300D0308A0127210730BA00BB
:100480002030B8005430AA004030AB00AE01AF01BC
:1004900063308A01AD200730BA001030B800543004
:1004A000AA004030AB000230A9005230B000B101C8
:1004B0008A0173200230A9005230B000B1018A01D4
:1004C0007920C5000430A9005230B000B1018A0182
:1004D0007920BC002508BD000130A9005230B000D1
:1004E000B1018A017920BE002508BF000230A900B1
:1004F0005230B000B1018A0173200230A90052309D
:10050000B000B1018A017920CC000230A90052303C
:10051000B000B1018A0173200230A9005230B0004E
:10052000B1018A017920CB000130A300F4308A01A7
:100530002721FE308A01032001308A010320523036
:100540008A01032058308A01032049088A010320C8
:1005500020308A0103200230A9004508A400A5012B
:100560000230B000B1018A01F8200130A9003C0836
:10057000A0003D08A100E830A2000330A3008A01DA
:100580007F21B2002108B3003208A4003308A5007F
:100590000230B000B1018A01F8202E308A01032018
:1005A0000330A9003C08A4003D08A5000230B000BB
:1005B000B1018A01F8202E308A0103200130A90000
:1005C0003E08A4003F08A5000230B000B1018A0136
:1005D000F8204D308A01032048308A0103207A3008
:1005E0008A0103208A150A129F22C8308A01262117
:1005F00064008A110A12871C182B64008A110A12DF
:10060000071D522B64008A110A12871D0E2B6400ED
:100610008A150A12071F3F288A01992A32308A0157
:10062000262164008A110A128719E22B8A010E2BF7
:100630000730BA002030B8005430AA004030AB0078
:10064000AE01AF012B308A01AD200730BA00103067
:10065000B8005430AA004030AB000130A90052303D
:10066000B000B1018A0173200230A9005230B000FD
:10067000B1018A017920C5000430A9005230B000D0
:10068000B1018A017920BC002508BD000130A90014
:100690005230B000B1018A017920BE002508BF00A8
:1006A0008A01992A4908A00072308A015A21B200B1
:1006B0003C08A0003D08A1001130A300F8308A01D9
:1006C0006221B4003208840034088A0178218A113A
:1006D0000A12031DA52B0730BA002030B800543091
:1006E000AA004030AB00AE01AF012D308A01AD2031
:1006F0000730BA001030B8005430AA004030AB00C8
:100700000130A9005230B000B1018A0173200230DB
:10071000A9005230B000B1018A017920C50004302F
:10072000A9005230B000B1018A017920BC0025082F
:10073000BD000130A9005230B000B1018A0179201A
:10074000BE002508BF008A01992AFE308A010320D5
:1007500001308A0103202A308A01032046308A01B1
:10076000032075308A01032065308A01032072302E
:100770008A01032061308A01032020308A0103208E
:1007800064308A01032065308A01032020308A0109
:10079000032062308A01032061308A0103206E3019
:1007A0008A01032064308A01032061308A0103201A
:1007B0002A308A0103200330A300E8308A01272170
:1007C0008A01992A0730BA002030B8005430AA00B4
:1007D0004030AB00AE01AF0176308A01AD2007306A
:1007E000BA001030B8005430AA004030AB000130DD
:1007F000A9005230B000B1018A0173200230A90073
:100800005230B000B1018A017920CC00FE308A015B
:10081000032001308A01032020308A010320203088
:100820008A01032020308A01032020308A0103201E
:1008300056308A0103204F308A0103204C308A0150
:10084000032055308A0103204D308A0103204530B2
:100850008A0103204E308A01032020308A010320C0
:1008600020308A01032020308A01032020308A01B1
:100870000320FE308A010320C0308A01032020308B
:100880008A0103202A308A01032020308A010320B4
:100890004E308A01032049308A01032056308A01F4
:1008A000032045308A0103204C308A0103202D307B
:1008B0008A01032020308A0103200230A9004C085D
:1008C000A400A5010230B000B1018A01F820203057
:1008D0008A0103202A308A01032064008A110A1247
:1008E000871C7E2C64008A110A12071D902C64005C
:1008F0008A110A12871DA22C8A016D2C64308A018C
:1009000026210730BA002030B8005430AA00403009
:10091000AB00AE01AF012B308A01AD208A01EF2B75
:1009200064308A0126210730BA002030B8005430E4
:10093000AA004030AB00AE01AF012D308A01AD20DE
:100940008A01EF2B64308A0126210730BA0020305B
:10095000B8005430AA004030AB00AE01AF01763091
:100960008A01AD20C8308A01262132308A01262131
:1009700064008A110A128719BF2C8A01B52C07302E
:10098000BA002030B8005430AA004030AB00AE01AD
:10099000AF0171308A01AD200730BA001030B800C5
:1009A0005430AA004030AB000130A9005230B000F2
:1009B000B1018A0173200230A9005230B000B101A8
:1009C0008A017920CB00FE308A01032001308A01A0
:1009D000032020308A01032020308A0103202030A8
:1009E0008A01032020308A01032053308A0103202A
:1009F00051308A01032055308A01032045308A0195
:100A000003204C308A01032043308A010320483000
:100A10008A01032020308A01032020308A0103202C
:100A200020308A01032020308A010320FE308A0111
:100A30000320C0308A01032020308A0103202A309D
:100A40008A01032020308A0103204E308A010320CE
:100A500049308A01032056308A01032045308A013B
:100A600003204C308A0103202D308A0103202030DE
:100A70008A0103200230A9004B08A400A50102301E
:100A8000B000B1018A01F82020308A0103202A3009
:100A90008A01032064008A110A12871C5B2D6400FE
:100AA0008A110A12071D6D2D64008A110A12871D12
:100AB0007F2D8A014A2D64308A0126210730BA0031
:100AC0002030B8005430AA004030AB00AE01AF0176
:100AD0002B308A01AD208A01CC2C64308A0126217A
:100AE0000730BA002030B8005430AA004030AB00C4
:100AF000AE01AF012D308A01AD208A01CC2C6430CB
:100B00008A0126210730BA002030B8005430AA00EC
:100B10004030AB00AE01AF0171308A01AD20C8306A
:100B20008A01262132308A01262164008A110A12A4
:100B300087199C2D8A01922D64004908723C8A1104
:100B40000A120319AA2D64004908003C8A110A12EE
:100B50000319342E64308A012621FE308A010320D5
:100B600001308A01032020308A0103202A308A01C3
:100B7000032052308A01032065308A01032070303F
:100B80008A01032065308A01032074308A01032022
:100B900069308A01032064308A0103206F308A01A2
:100BA000032072308A01032020308A0103204F3055
:100BB0008A0103204E308A0103202A308A01032053
:100BC00020308A010320FE308A010320C0308A01D0
:100BD000032020308A01032020308A0103202030A6
:100BE0008A01032028308A01032044308A0103202F
:100BF0006F308A01032077308A0103206E308A012A
:100C000003203D308A0103204F308A010320463003
:100C10008A01032046308A01032029308A010320FB
:100C200020308A01032020308A01032020308A01ED
:100C300003207230C9003C08A0003D08A10011301B
:100C4000A300F8308A0165218A110A12031DDC2EE7
:100C500064008A110A12071DB62E64008A110A1256
:100C6000871D262F8A01AA2D64308A012621FE3095
:100C70008A01032001308A01032020308A010320E9
:100C80002A308A01032052308A01032065308A010C
:100C9000032070308A01032065308A0103207430FC
:100CA0008A01032069308A01032064308A0103200D
:100CB0006F308A01032072308A01032020308A01BC
:100CC00003204F308A01032046308A01032046303A
:100CD0008A0103202A308A01032020308A01032060
:100CE000FE308A010320C0308A01032020308A01AF
:100CF000032020308A01032020308A010320203085
:100D00008A01032028308A01032055308A010320FC
:100D100070308A0103203D308A0103204F308A0160
:100D200003204E308A01032029308A01032020301D
:100D30008A01032020308A01032020308A01032009
:100D400020308A01032020308A01032020308A01CC
:100D50000320C90164008A110A12871CB62E6400A0
:100D60008A110A12871D262F8A01342E0730BA00F5
:100D70002030B8005430AA004030AB00AE01AF01C3
:100D800073308A01AD200730BA001030B8005430FB
:100D9000AA004030AB008A015220CA0064004A0811
:100DA000533C8A110A120319AA2D64004A08413CD7
:100DB0008A110A120319342EFE308A0103200130F1
:100DC0008A0103202A308A01032046308A01032049
:100DD00075308A01032065308A01032072308A0150
:100DE000032061308A01032020308A01032064300F
:100DF0008A01032065308A01032020308A01032004
:100E000042308A01032061308A0103206E308A015A
:100E1000032064308A01032061308A0103202A30D4
:100E20008A0103200330A300E8308A01272107301C
:100E3000BA002030B8005430AA004030AB00AE01F8
:100E4000AF0173308A01AD208A01342E64008A110B
:100E50000A1287192D2F8A01262F64008A110A127F
:100E60004818372F64008A110A12481CB72FFE3029
:100E70008A01032001308A01032020308A010320E7
:100E80002A308A01032050308A01032061308A0110
:100E900003206E308A01032074308A010320613000
:100EA0008A0103206C308A0103206C308A01032000
:100EB00061308A01032020308A0103204F308A01EB
:100EC00003204E308A0103202A308A01032020307B
:100ED0008A01032020308A010320FE308A0103208A
:100EE000C0308A01032020308A01032020308A018B
:100EF000032028308A01032044308A0103206F3008
:100F00008A01032077308A0103206E308A01032092
:100F10003D308A0103204F308A01032046308A0188
:100F2000032046308A01032029308A010320203023
:100F30008A01032020308A01032020308A01032007
:100F400020308A01032007148316071083124814E7
:100F500064008A110A12071DB72F64008A150A124D
:100F6000871D372864308A0126218A01372FFE30F9
:100F70008A01032001308A01032020308A010320E6
:100F80002A308A01032050308A01032061308A010F
:100F900003206E308A01032074308A0103206130FF
:100FA0008A0103206C308A0103206C308A010320FF
:100FB00061308A01032020308A0103204F308A01EA
:100FC000032046308A01032046308A0103202A305C
:100FD0008A01032020308A010320FE308A01032089
:100FE000C0308A01032020308A01032020308A018A
:100FF000032020308A01032020308A01032028307A
:101000008A01032055308A01032070308A010320B1
:101010003D308A0103204F308A0103204E308A017F
:10102000032029308A01032020308A010320203048
:101030008A01032020308A01032020308A01032006
:1010400020308A01032007108316071083124810EE
:1010500064008A110A12871C372F64008A150A124D
:10106000871D372864308A0126218A01B72F640042
:101070008A110A128719992A8A150A1237286400D8
:101080004A08413C8A150A1203194D2864004A088F
:10109000533C8A150A12031991288A150A12D52081
:1010A0008A150A120E21FE308A010320C0308A01FF
:1010B000032020308A01032020308A0103202030C1
:1010C0008A01032020308A0103202A308A0103206C
:1010D0002A308A01032020308A01032054308A01FB
:1010E000032058308A01032020308A0103202A304F
:1010F0008A0103202A308A01032020308A0103203C
:1011000020308A01032020308A01032020308A0108
:10111000032064008A150A12871DB0298A150A1255
:1011200068218A150A12D5208A150A120E21FE306E
:101130008A010320C0308A0103202A308A0103205B
:101140002A308A01032020308A01032054308A018A
:10115000032058308A01032020308A0103202D30DB
:101160008A01032036308A01032030308A010320AF
:1011700030308A0103204B308A01032048308A0135
:1011800003207A308A01032020308A0103202A308C
:101190008A0103202A308A01032064008A150A127A
:1011A000871DB0298A150A1268210730BA0020303D
:1011B000B8005430AA004030AB00AE01AF0174302B
:1011C0008A01AD200730BA001030B8005430AA00B0
:1011D0004030AB000130A9005230B000B1018A01AB
:1011E00073200230A9005230B000B1018A01792089
:1011F000C5000430A9005230B000B1018A01792045
:10120000BC002508BD000130A9005230B000B1017A
:101210008A017920BE002508BF000800FE308A013F
:10122000032001308A01032054308A010320583002
:101230008A01032049088A01032020308A01032003
:101240000230A9004508A400A5010230B000B10198
:101250008A01F8200130A9003C08A0003D08A10047
:10126000E830A2000330A3008A017F21B2002108E8
:10127000B3003208A4003308A5000230B000B10169
:101280008A01F8202E308A0103200330A9003C088F
:10129000A4003D08A5000230B000B1018A01F82089
:1012A0002E308A0103200130A9003E08A4003F0827
:1012B000A5000230B000B1018A01F8204D308A014A
:1012C000032048308A0103207A308A010320080075
:1012D00064008A150A12071B732964308A012621CB
:1012E0008A150A123F280730BA002030B80054305F
:1012F000AA004030AB00AE01AF0172308A01AD20D0
:101300000730BA001030B8005430AA004030AB00AB
:101310000130A9005230B000B1018A0173200230BF
:10132000A9005230B000B1018A017920C500043013
:10133000A9005230B000B1018A017920BC00250813
:10134000BD000130A9005230B000B1018A017920FE
:10135000BE002508BF0032308A0126218A01992A61
:1013600064308A01262164008A150A12871DB0297B
:101370000730BA002030B8005430AA004030AB002B
:10138000AE01AF0164308A01AD200730BA001030E1
:10139000B8005430AA004030AB000130A9005230F0
:1013A000B000B1018A0173200230A9005230B000B0
:1013B000B1018A017920C400FE308A010320013086
:1013C0008A01032020308A01032020308A01032073
:1013D00020308A01032020308A01032020308A0136
:1013E00003204D308A01032049308A010320433015
:1013F0008A01032052308A0103204F308A010320E2
:1014000020308A01032020308A01032020308A0105
:10141000032020308A01032020308A01032020305D
:101420008A010320FE308A010320C0308A01032094
:1014300020308A0103202A308A01032020308A01CB
:1014400003204E308A01032049308A0103205630A0
:101450008A01032045308A0103204C308A01032091
:101460002D308A01032020308A0103200230A90098
:101470004408A400A5010230B000B1018A01F8209F
:1014800020308A0103202A308A01032064308A0137
:10149000262164008A150A12871C5B2A64008A15BB
:1014A0000A12071D6E2A64008A150A12871D812AF6
:1014B0008A150A12462A64308A0126210730BA00AA
:1014C0002030B8005430AA004030AB00AE01AF016C
:1014D0002B308A01AD208A150A12C52964308A0191
:1014E00026210730BA002030B8005430AA0040301E
:1014F000AB00AE01AF012D308A01AD208A150A1272
:10150000C52964308A0126210730BA002030B8008E
:101510005430AA004030AB00AE01AF0164308A0104
:10152000AD2064308A01262132308A0126216400F0
:101530008A150A1287193F288A150A12942AFE3042
:101540008A01032040308A0103200830A9000230BC
:10155000B000B10100308A01F02000308A01032080
:101560000630A9000230B000B10110308A01F0202D
:1015700000308A01032000308A0103200630A900D0
:101580000230B000B10114308A01F02000308A012D
:10159000032000308A0103200630A9000230B00089
:1015A000B10115308A01F02000308A010320073094
:1015B000BA002030B8005430AA004030AB00AE0171
:1015C000AF016E308A01AD200730BA001030B8008C
:1015D0005430AA004030AB000130A9005230B000B6
:1015E000B1018A0173200330A9005230B000B1016B
:1015F0008A017920C3004308863CB2000030031CF6
:10160000FF3EB3003208A6003308A7004C30A2000A
:10161000A3018A019B21B2002508B3003208A00073
:101620003308A1000A30A200A3018A017F21B20081
:101630002108B3001E303202C0000030031C013EFE
:101640003302C1006400463043028A150A12031CAB
:10165000852B4008A0004108A1001330A200A3017F
:101660008A017F21C2001830A000A10142088A012E
:101670004821B2002108B3003208A0003308A100BD
:101680000330A200A3018A017F21C6001830A00008
:10169000A10142088A014821B2002108B3003208A2
:1016A000A0003308A1000330A200A3018A017F211A
:1016B0002408C700FE308A010320C0308A010320BD
:1016C0002D308A0103200330A9004308A400A5019E
:1016D0000230B000B1018A01F82064308A01032091
:1016E00042308A0103206D308A01032020308A01B4
:1016F00003204608A9000230B000B10103308A017E
:10170000F02047088A0103200800FE308A010320E8
:10171000C0308A01032020308A0103204E308A0124
:10172000032069308A01032076308A010320653066
:101730008A0103206C308A01032020308A010320B3
:101740002A308A01032020308A0103204F308A0189
:10175000032056308A01032045308A01032052308D
:101760008A01032020308A0103202A308A010320C5
:0817700020308A01032008006B
:02400E00753DFE
:00000001FF
